:060000001F308A000028F9
:10300000031383161F3099000D2803138312A101A7
:1030100083168B138B1B052812288312A101A11480
:103020008316181518080439223898001F308A00B2
:1030300007178717D7308100831290309800C60198
:10304000C501A001C00140148A26EF25FA25A01C65
:103050002F28A11C2F285C233C21201D7C28A01791
:103060008120A013201B3728A0187C282F28212678
:103070005C2360210008A721AC00031938285730D1
:103080002C02031D4528CE20382852302C02031D67
:103090004B28A4203828840A0008031D7A283F30D2
:1030A0002C02031D55287C25382855302C02031D81
:1030B00066288722201D3828A01962285B25F52064
:1030C000FA253828302184231C25382844302C0246
:1030D000031D6C28BD21382851302C02031D742893
:1030E000A0187C28FA25382856302C02031D7A288F
:1030F000FA25382899243828A01C382844268A0123
:1031000003282013A228503091216130912173307F
:1031100091219121773091216F309121723091214D
:10312000643091213E30912160212208F62700026F
:10313000031DA32800080319A228A219A328A20A84
:10314000840A952820170800840A20300002031DF5
:10315000B528840AA0119821A800A019B528000854
:10316000031DB5281624B720080099240800280854
:10317000C320203091213D3091212030912127081A
:10318000C32084230800B900F039B000300EE527D1
:10319000912139080F39E52791210800840A203050
:1031A0000002031DF328840AA0119821A019F32816
:1031B000A70020300002031DF328840A40300002DB
:1031C000031DF328840A20300002031DF328840A1B
:1031D0009821A800A019F3280008031DF328F6235E
:1031E0001624B7200800992408001F30A500C53018
:1031F000A6003430A30047256021A20A0008A400DD
:103200009023000803190800A60A840AA20AA21A39
:103210008001FE286400201018191229981C142916
:10322000181218161A0808008C1E080020141A0814
:10323000C3000A3C031920104308080081010B1148
:103240000A21201C242908000B1D2029A11908008F
:10325000C50A0319C60AC61E0800A0187C28080063
:10326000A1151E21201830291E21201830291E21C9
:1032700020183029A11108002011A1151A30BE0014
:103280000F30AB0020309121AB0B42293C30912113
:103290001030AB0008309121AB0B4A290F30AB0046
:1032A0001E2120185C29BE0B50291A30BE00233085
:1032B0009121AB0B50295D292015A1118423080011
:1032C00050308400C601C5011E21201C642908302D
:1032D0004302031D7A295030040203196229840332
:1032E0000830211C91212030211C91210830211C03
:1032F000912162290D30430203198A294308800075
:10330000A01B2A30211C91217F30040203198A2935
:10331000840A6229211C84238001A2015030840088
:10332000080081010B1164000C1E9329990008000C
:103330000008A7217226A0190800B000B00E840A68
:103340000008A7217226B0043008840A0800C300D0
:103350007B3043020318B32961304302031CB329B5
:1033600020304302080043080800E0233F302302D6
:10337000031D0800FF3024020800A011FA25A01C3C
:103380000800A5010330A600B101B521031DCF2916
:10339000A60A0319A50A2224A01DC429EA29250882
:1033A000BA002608BB00B10A2608AF00A60A031916
:1033B000A50A2F082606F839031DE4292224A0199E
:1033C000E929B521031DD32923222224A019EA29A2
:1033D000C4292322FA21A0113A3091210030C320C0
:1033E0000030C3200030C3200130C320FF30C32091
:1033F00084230800A8014230BF003A3091211030E8
:10340000B200B6000310B60CC3200310280D031839
:103410003F143F08B207C3200310280DB207C32092
:103420000301C32016242708B207C3200301C320C9
:10343000A80AB60B122AB209320AC320842328082C
:10344000031DFD2908003A08A5003B08A6003A30F4
:1034500091210310310DB200C320260D250DB207B6
:10346000C3200310260DB207C3200301C320E023AD
:10347000A60A0319A50A2408B207C3202308B20725
:10348000C320B10B372AB209320AC32084230800B3
:103490004530912172309121613091217330912119
:1034A000693091216E309121673091218423A010E1
:1034B000A5010330A6003F30A300FF30A4009023F5
:1034C000A0190800A60A031D682AA50A2330912125
:1034D0002224A01D5F2AA0111F30A500C530A60020
:1034E0003430A300A4019023A0190800A60AE530F7
:1034F0002602031D732AFF30A800FF30A700F62321
:10350000A0190800A80B7F2AF62384230800A01125
:103510002011B301B401B5014130912172309121E4
:103520006530912120309121793091216F309121A6
:103530007530912120309121733091217530912186
:1035400072309121653091213F30912120309121BD
:103550005B309121793091212F3091214E30912192
:103560005D3091213E30912160210008A721593C16
:10357000031D0800840A0008031D080020154822C6
:10358000A0190800523091216530912161309121BC
:1035900064309121793091218423211621146021F6
:1035A0002110B30A0A303302031CDE2AB301B40A25
:1035B0000A303402031CDE2AB401B50A00083A3C82
:1035C000031D362B840A9821A0190800B100B2000F
:1035D0000310310CB100B8009821A0190800A50013
:1035E000B2079821A0190800A600B2070310A50C85
:1035F000A60C9821A0190800B700B207B708031D50
:10360000322B0408C200B1080319102B9821A0190D
:103610000800B2079821A0190800B207B103032BD4
:103620009821A0190800B207031D522B42088400FC
:10363000B808031D1E2B23309121CE2A9821A40007
:103640009821A3002224A0193F24A0190800A01E3D
:103650009023A01A5623A0190800A60A0319A50A48
:10366000B803182B842337030319392BA015D5244D
:1036700008009821A0190800B207031D522B21123F
:103680004708A3004808A400A5010330A600902322
:10369000EF25A0180800A0156523B301B401B501FA
:1036A000B30A0800A0158423EF2408002408A7000B
:1036B0002608A800F62308005030912149309121B6
:1036C000433091213E3091210800303091219121E9
:1036D0009121333091216830912120309121213086
:1036E00091213D30912120309121673091216F301F
:1036F0009121743091216F309121203091215830E7
:1037000091219121842308000A3091210D309121CB
:103710000800203091212D30912120309121080086
:10372000201264002508031DA02B03302602031D70
:10373000A02B211EA02B2308C7002408C8000800C6
:10374000250803178F000313260803178D000313A2
:10375000230803178E000313240803178C00831615
:103760008C170C1555308D00AA308D008C14FF3F3E
:10377000FF3FFF3FFF3FFF3FFF3FFF3FFF3FFF3F59
:10378000FF3FFF3FFF3FFF3FFF3FFF3FFF3F000087
:1037900000000C110C140000000083120E0803132B
:1037A0002302031DD92B03170C080313240203194A
:1037B0000800201ADD2B2016A02B7C24A015080061
:1037C0006400250803178F000313260803178D00D4
:1037D00083168C170C140000000083120E080313CC
:1037E000A30003170C080313A40008000D122808F7
:1037F00003178D000313270803178C0083168C13FF
:103800000C1555308D00AA308D008C1483120313D3
:1038100064000D1E082C031783160C110C14831260
:103820000C0803132702031D8A24080064002808DB
:1038300003178D0083168C130C1483120C080313CA
:10384000A7000800A01203012502031D332C030169
:10385000260203193D2C0130260203193D2C0230AB
:10386000260203193D2C18302502031C08002508E8
:10387000213C031D3D2CA0160800A01508004D306A
:103880009121653091216D3091216F3091217230FD
:103890009121793091212030912170309121723025
:1038A00091216F30912174309121653091216330E5
:1038B000912174309121693091216F3091216E30C6
:1038C000912102251025080020309121703091218E
:1038D000723091216F3091216730912172309121A6
:1038E000613091216D3091219121693091216E30AB
:1038F0009121673091210800463091214C3091216F
:103900004130912153309121483091216424022586
:1039100010250800453091219121503091215230DD
:1039200091214F3091214D30912164248423A015A1
:103930000800C424633091216F3091216D309121B2
:103940009121613091216E30912164309121842345
:1039500008004E3091216F3091216E3091212D3031
:1039600091214830912145309121583091212030CA
:103970009121633091216830912161309121723021
:103980009121022584230800493091216E30912134
:1039900076309121613091216C30912169309121F3
:1039A00064309121203091210800C424723091218B
:1039B00065309121633091216F30912172309121D6
:1039C00064309121203091217430912179309121FE
:1039D0007030912165309121022584230800433005
:1039E00091216830912165309121633091216B30B4
:1039F000912173309121753091216D3091210225F3
:103A0000842308002030912165309121723091216A
:103A100091216F3091217230912120309121080045
:103A200040309121203091212508C3202608C32051
:103A300068309121842308004C3091216930912114
:103A40006E30912165309121203091216E3091218D
:103A5000753091216D309121623091216530912135
:103A60007230912120309121A012350803193B2D8D
:103A7000A016E52791213408A01A402D0319422DE4
:103A8000E52791213308E52791218423080045305B
:103A900091216E30912174309121653091217230E5
:103AA0009121203091216130912120309121BA253E
:103AB0003E309121080055309121703091216C30B9
:103AC00091216F309121613091216430912120301A
:103AD0009121733091217530912163309121912191
:103AE000653091217330912166309121753091219B
:103AF0006C30912184230800C001C0148A265B2603
:103B000084235530912189235530912170309121A2
:103B10006C3091216F30912161309121643091217D
:103B20005B26743091216F309121CF254430912153
:103B30008923443091216F309121773091216E306B
:103B400091216C3091216F3091216130912164304D
:103B500091215B2666309121723091216F30912145
:103B60006D309121CF25C00140158A265B26BA25EC
:103B700084230800723091216530912176309121A3
:103B80002030912173309121743091217230912134
:103B9000693091216E3091216730912108002030E9
:103BA000912170309121723091216F3091216730D5
:103BB000912172309121613091216D30912120301D
:103BC00091216D309121653091216D3091216F30BF
:103BD0009121723091217930912184230800A01025
:103BE000A5010330A600E02323083839283A031939
:103BF000A0140800A01C072EC527FF390319192E91
:103C0000C00140168A26C001C0158A261F2E4E30DC
:103C100091216F3091215B266C3091216F30912181
:103C2000613091216430912165309121643091217E
:103C30001F2E4E3091216F3091215B26BA258423AF
:103C4000080038263F3091212030912166309121A3
:103C50006F30912172309121203091216830912173
:103C6000653091216C3091217030912184230800BE
:103C70005030912172309121653091217330912122
:103C800091212030912108004A30912175309121F5
:103C90006D30912170309121693091216E309121E8
:103CA0006730912120309121743091216F30912122
:103CB0005B268423080020309121753091217330D8
:103CC0009121653091217230912120309121633012
:103CD00091216F3091216430912165309121203004
:103CE00091210800AF003030AF02031C872E0A304C
:103CF0002F02031C852E1130AF02031C872E0630C5
:103D00002F020318872E0A30AF072F080800A015CE
:103D1000A9240034AF012F0840188F27C01862274C
:103D200040190327C019C427401A5027FF39031927
:083D300008009121AF0A8B2E5F
:0A3E06008207573420342D34203495
:103E100057347234693474346534203474346F34F4
:103E2000203445344534503452344F344D342C34DE
:103E30002034223457342034443444342034403441
:103E400020344134413422340A340D345234203485
:103E50002D34203452346534613464342034663473
:103E600072346F346D342034453445345034523418
:103E70004F344D342C3420342234523420344134E5
:103E8000413422340A340D34563420342D34203455
:103E900044346934733470346C34613479340034AC
:103EA0008207433475347234723465346E3474343A
:103EB000203469346D3461346734653420343D34E2
:103EC0002034003482073F3420342D3420344434ED
:103ED0006934733470346C3461347934203474341C
:103EE00068346934733420346C3469347334743412
:103EF0000A340D34513420342D3420345134753487
:103F000069347434203461346E34643420346A3457
:103F100075346D347034203474346F340034820757
:103F20001B345B3432344A3438344B34203450340C
:103F3000493443344C344F3441344434453452349E
:103F40002034763431342E3431340A340D34433451
:103F50006F3470347934723469346734683474344B
:103F600020345234693463346B3420344634613441
:103F700072346D3465347234203431343934393428
:103F800039340A340D3400348207003400340034EC
:103F90000034003400340034003400340034003481
:103FA0000034003400340034003400340034003471
:103FB0000034003400340034003400340034003461
:103FC000003400340034003400348207303431349B
:103FD0003234333434343534363437343834393495
:103FE00041344234433444344534463482074834FF
:103FF00065346C346C346F343134323433340034DF
:02400E00723FFF
:00000001FF
